:100000000828FF3FFF3FFF3F0C2C9F2A8A018200F8
:10001000FF30A200FF30A300BE220A306B23241160
:10002000BE230330B522323084230330B522323070
:1000300084230330B522323084233230A922283081
:10004000A9222312DA23A312D9232313D82392231C
:100050002216DB23A317D7232214DF23A214DE23C7
:10006000A6010F30A700A8010F30A900A0113C3055
:10007000B6006E30B5004621BD2059218F220030D8
:1000800087225030A1225930A1223230A1224330A0
:10009000A1225330A1225930A1222030A122543074
:1000A000A1225230A1225830A1223230A1224D305B
:1000B000A1220D308B225230A1225830A12265207E
:1000C0009D207D20EB205F286428861B7228A019C4
:1000D0007128A01559210D308B225430A12258309F
:1000E000A1227C28A01D7C28A01159210D308B2233
:1000F0005230A1225830A1220800290828020318F2
:100100008A28851C8A28A80A28082902031D89280C
:100110008C208B28A8010800CC2020199C28B70827
:10012000031D99283808013C031D99280130380225
:10013000B80001303702B700BD282708260203188F
:10014000AA28051CAA28A60A26082702031DA928F2
:10015000AC20AB28A6010800CC20A018BC28380889
:10016000BD003708BE00BF010130C000F1224108C8
:10017000B8004208B700BD2008003608BD003508A9
:10018000BE003808BF003708C000F1224108AB00AC
:100190004208AA00512159293D302B02031CDA28BC
:1001A000FE302A02031CDA28A0143D30AB00FE30DA
:1001B000AA00DB28A0102B083C3C031CE9282A08D5
:1001C0006E3C031CE92820153C30AB006E30AA00C1
:1001D000EA28201108002B08AF002A08AE002E08DC
:1001E0002E3C0318FA2804302F02B1002E302E02C4
:1001F000B00010292E082E3C031D032904302F02C5
:10020000B100B00110292E302E020318102904303D
:100210002F02BD0001303D02B1002E302E02B00091
:100220003008BD003108BE006430BF00C001CA22E2
:100230003D08B0003E08B1004108AC004208AD00E6
:100240002D08C0002C085D223D08B2003E08B30016
:100250003F08B40000308B220430BD003308BE00DC
:10026000203005230430BD003408BE003030102398
:100270002E30A1220430BD003008BE0030302423CF
:100280004D30A1224830A1227A30A12A0130BD0090
:10029000AF233E08B7000230BD00AF233E08B800D0
:1002A00008000130BD00370897230230BD00380830
:1002B000972BA01D89292B08BA002A08B9003908F4
:1002C0002E3C03186A2904303A02BC002E30390251
:1002D000BB00802939082E3C031D732904303A02E3
:1002E000BC00BB0180292E3039020318802904305C
:1002F0003A02BD0001303D02BC002E303902BB0085
:100300001430BD003C08BE003B08BF0045309221C0
:1003100091291430BD002B08BE002A08BF004530CB
:1003200092210800C0005B222513BA232512BC23AA
:10033000A512BB235B222512BC230830C100251364
:10034000BD1FA3292517BA235B222516BC235B22D8
:100350002512BC235B220310BD0DC10B9F295B221C
:10036000A516BB235B225B220830C10025133F1C6E
:10037000BA292517BA235B222516BC235B22251236
:10038000BC235B220310BF0CC10BB6295B225B228E
:100390005B225B220830C10025133E1CD0292517A3
:1003A000BA235B222516BC235B222512BC235B22C9
:1003B0000310BE0CC10BCC295B225B225B225B22AB
:1003C0000830C1002513C01FE6292517BA235B2278
:1003D0002516BC235B222512BC235B220310C00D13
:1003E000C10BE2295B22A512BB235B225B22943066
:1003F000C100C2010330C300C4010830C500251389
:10040000C11F032A2517BA235B222516BC235B22B2
:100410002512BC235B220310C10DC50BFF295B22F3
:10042000A516BB235B225B220830C5002513C21F23
:100430001A2A2517BA235B222516BC235B22251214
:10044000BC235B220310C20DC50B162A5B225B2264
:100450005B225B220830C5002513C31F302A2517F5
:10046000BA235B222516BC235B222512BC235B2208
:100470000310C30DC50B2C2A5B225B225B225B227F
:100480000830C5002513C41F462A2517BA235B224E
:100490002516BC235B222512BC235B220310C40D4E
:1004A000C50B422A5B22A512BB232512BC232513B0
:1004B000BA235B225B2A0530902BC100BD01BE012F
:1004C000BF011030C2003F0877224308BF003E083A
:1004D00077224308BE003D0877224308BD00C10DC6
:1004E000C00DBF0DBE0DBD0DC20B632A0800C300B9
:1004F0004308033EC400C41D7F2A4408C3004308C8
:10050000303EC400C41F862A4408C3000800BD0052
:100510003D08C03EA92ABD003D08803EA92A0830FA
:10052000A9220130A922C83084230230A922C83070
:1005300084230630A9220C30A922C830842B21083C
:10054000C500C5002415BE23450E0F39B522450848
:10055000B52ABE002411BE233E0E0F39B5228230CB
:1005600084233E08B5228230842BC600A415BD2307
:100570004608BF23A411BD23FA30902B0030BF23BF
:100580002411BE23A411BD230030CE232211DD236C
:10059000A211DC2BC200C101C2010130C300C401A1
:1005A000C01BD82A0310C30DC40DBF0DC00DD02A27
:1005B0003F083D02C5000030031C013040073E02E9
:1005C000031CE92ABE004508BD004308C1074408D2
:1005D000C2070310C00CBF0CC40CC30C031CD82AE8
:1005E0000800C2003E08FF3CC30040084302031855
:1005F000FE2A3D083F07013EC100012B3D083F0791
:10060000C1003E084007C2000800BF003D08C2000C
:100610003E080F39C3003F084C234408BF000800C0
:10062000BF003D08C2003E0E0F39C3003F084C23F7
:100630004408BF003D08C2003E080F39C3003F0810
:100640004C234408BF000800BF003E08C2006430CD
:10065000C300EC23C0004008BE003D08C2003E08B5
:10066000C5000A30C600FB23C4004408C3003F088D
:100670004C234408BF003E08C2000A30C300EC23EC
:10068000C1004108BE003D08C2003E08C3003F084B
:100690004C234408BF000800C400C308031D582BA6
:1006A000C4080319572B4408A100420A06206A2BEC
:1006B0000A3043020318622B4308303EA100420A6D
:1006C0000620682B0A304302413EA100420A062060
:1006D0003030C4000800A6002608A7006430A80037
:1006E0000130722BA900FF30AA002808AC002708AF
:1006F000AB001A302A0703187A2BAB0B792BAC0B03
:10070000772BA90B752B0800BF003F08C000C0085D
:10071000031D8B2B8F2B0A309023C003872B0800DF
:10072000C700080007309F00E6231F13E92BBE0017
:10073000831203133E0883169A0083123D08831622
:100740009B001C158B138B1355309D00AA309D0008
:100750009C149C18A92B1C118B1783120800BE0037
:10076000831203133D0883169B001C141A0883127E
:10077000BE000800C82BC82BC82BCB2BCB2BC70027
:1007800047080F39C8002508F0394804A500C82BD0
:10079000250886000800240885000800A600260811
:1007A0000F39A7002308F0392704A300E02BE02B22
:1007B000E02BE02BE02BE32BE32BE32BE32BE32BD2
:1007C000230866000800220865000800831603134A
:1007D0000800831203130800C300C3080319F92B90
:1007E000430842020318F52BF92B43084202C200CA
:1007F000F02B42080800C600C701C60803190A2CDE
:10080000460845020318052C0A2C46084502C50077
:10081000C70A002C470808000430A1000800FF3F69
:10082000FF3FFF3FFF3FFF3FFF3FFF3FFF3FFF3FD8
:10083000FF3FFF3FFF3FFF3FFF3FFF3FFF3FFF3FC8
:10084000FF3FFF3FFF3FFF3FFF3FFF3FFF3FFF3FB8
:10085000FF3FFF3FFF3FFF3FFF3FFF3FFF3FFF3FA8
:02400E00623F0F
:10420000FF00FF00FF00FF00FF00FF00FF00FF00B6
:10421000FF00FF00FF00FF00FF00FF00FF00FF00A6
:10422000FF00FF00FF00FF00FF00FF00FF00FF0096
:10423000FF00FF00FF00FF00FF00FF00FF00FF0086
:10424000FF00FF00FF00FF00FF00FF00FF00FF0076
:10425000FF00FF00FF00FF00FF00FF00FF00FF0066
:10426000FF00FF00FF00FF00FF00FF00FF00FF0056
:10427000FF00FF00FF00FF00FF00FF00FF00FF0046
:10428000FF00FF00FF00FF00FF00FF00FF00FF0036
:10429000FF00FF00FF00FF00FF00FF00FF00FF0026
:1042A000FF00FF00FF00FF00FF00FF00FF00FF0016
:1042B000FF00FF00FF00FF00FF00FF00FF00FF0006
:1042C000FF00FF00FF00FF00FF00FF00FF00FF00F6
:1042D000FF00FF00FF00FF00FF00FF00FF00FF00E6
:1042E000FF00FF00FF00FF00FF00FF00FF00FF00D6
:1042F000FF00FF00FF00FF00FF00FF00FF00FF00C6
:00000001FF
